 jconsole

 Timestamp is 6710e06f (Thu Oct 17 10:01:19 2024)

 Preferred load address is 00400000

 Start         Length     Name                   Class
 0001:00000000 00000de8H .text$mn                CODE
 0002:00000000 000000f0H .idata$5                DATA
 0002:000000f0 00000008H .00cfg                  DATA
 0002:000000f8 00000004H .CRT$XCA                DATA
 0002:000000fc 00000004H .CRT$XCAA               DATA
 0002:00000100 00000004H .CRT$XCZ                DATA
 0002:00000104 00000004H .CRT$XIA                DATA
 0002:00000108 00000004H .CRT$XIAA               DATA
 0002:0000010c 00000004H .CRT$XIAC               DATA
 0002:00000110 00000004H .CRT$XIZ                DATA
 0002:00000114 00000004H .CRT$XPA                DATA
 0002:00000118 00000004H .CRT$XPZ                DATA
 0002:0000011c 00000004H .CRT$XTA                DATA
 0002:00000120 00000008H .CRT$XTZ                DATA
 0002:00000124 00000000H .gfids$y                DATA
 0002:00000128 00000218H .rdata                  DATA
 0002:00000340 00000000H .rdata$CastGuardVftablesA DATA
 0002:00000340 00000000H .rdata$CastGuardVftablesC DATA
 0002:00000340 00000004H .rdata$sxdata           DATA
 0002:00000344 00000064H .rdata$voltmd           DATA
 0002:000003a8 0000031cH .rdata$zzzdbg           DATA
 0002:000006c4 00000004H .rtc$IAA                DATA
 0002:000006c8 00000004H .rtc$IZZ                DATA
 0002:000006cc 00000004H .rtc$TAA                DATA
 0002:000006d0 00000008H .rtc$TZZ                DATA
 0002:000006d8 0000003cH .xdata$x                DATA
 0002:00000714 00000000H .edata                  DATA
 0002:00000714 000000b4H .idata$2                DATA
 0002:000007c8 00000014H .idata$3                DATA
 0002:000007dc 000000f0H .idata$4                DATA
 0002:000008cc 000004e6H .idata$6                DATA
 0003:00000000 00000040H .data                   DATA
 0003:00000040 0000037cH .bss                    DATA
 0004:00000000 00000060H .rsrc$01                DATA
 0004:00000060 00000320H .rsrc$02                DATA

  Address         Publics by Value              Rva+Base       Lib:Object

 0000:00000000       ___AbsoluteZero            00000000     <absolute>
 0000:00000000       ___arm64x_extra_rfe_table  00000000     <absolute>
 0000:00000000       ___arm64x_extra_rfe_table_size 00000000     <absolute>
 0000:00000000       ___arm64x_native_entrypoint 00000000     <absolute>
 0000:00000000       ___arm64x_redirection_metadata 00000000     <absolute>
 0000:00000000       ___arm64x_redirection_metadata_count 00000000     <absolute>
 0000:00000000       ___dynamic_value_reloc_table 00000000     <absolute>
 0000:00000000       ___enclave_config          00000000     <absolute>
 0000:00000000       ___guard_check_icall_a64n_fptr 00000000     <absolute>
 0000:00000000       ___guard_eh_cont_count     00000000     <absolute>
 0000:00000000       ___guard_eh_cont_table     00000000     <absolute>
 0000:00000000       ___guard_fids_count        00000000     <absolute>
 0000:00000000       ___guard_fids_table        00000000     <absolute>
 0000:00000000       ___guard_iat_count         00000000     <absolute>
 0000:00000000       ___guard_iat_table         00000000     <absolute>
 0000:00000000       ___guard_longjmp_count     00000000     <absolute>
 0000:00000000       ___guard_longjmp_table     00000000     <absolute>
 0000:00000000       ___hybrid_auxiliary_delayload_iat 00000000     <absolute>
 0000:00000000       ___hybrid_auxiliary_delayload_iat_copy 00000000     <absolute>
 0000:00000000       ___hybrid_auxiliary_iat    00000000     <absolute>
 0000:00000000       ___hybrid_auxiliary_iat_copy 00000000     <absolute>
 0000:00000000       ___hybrid_code_map         00000000     <absolute>
 0000:00000000       ___hybrid_code_map_count   00000000     <absolute>
 0000:00000000       ___hybrid_image_info_bitfield 00000000     <absolute>
 0000:00000000       ___x64_code_ranges_to_entry_points 00000000     <absolute>
 0000:00000000       ___x64_code_ranges_to_entry_points_count 00000000     <absolute>
 0000:00000001       ___safe_se_handler_count   00000001     <absolute>
 0000:00000100       ___guard_flags             00000100     <absolute>
 0000:00000000       ___ImageBase               00400000     <linker-defined>
 0001:00000000       _WinMain@16                00401000 f   main.obj
 0001:000000e5       ___local_stdio_printf_options 004010e5 f i main.obj
 0001:000000eb       __vfprintf_l               004010eb f i main.obj
 0001:0000010f       _printf                    0040110f f i main.obj
 0001:0000012d       _JLI_MemAlloc              0040112d f   jli:jli.dll
 0001:00000133       _JLI_GetStdArgs            00401133 f   jli:jli.dll
 0001:00000139       _JLI_GetStdArgc            00401139 f   jli:jli.dll
 0001:0000013f       _JLI_CmdToArgs             0040113f f   jli:jli.dll
 0001:00000145       _JLI_Launch                00401145 f   jli:jli.dll
 0001:0000038c       _WinMainCRTStartup         0040138c f   MSVCRT:exe_winmain.obj
 0001:000003da       ___scrt_acquire_startup_lock 004013da f   MSVCRT:utility.obj
 0001:0000040c       ___scrt_initialize_crt     0040140c f   MSVCRT:utility.obj
 0001:00000445       ___scrt_initialize_onexit_tables 00401445 f   MSVCRT:utility.obj
 0001:000004cc       ___scrt_is_nonwritable_in_current_image 004014cc f   MSVCRT:utility.obj
 0001:00000560       ___scrt_release_startup_lock 00401560 f   MSVCRT:utility.obj
 0001:0000057d       ___scrt_uninitialize_crt   0040157d f   MSVCRT:utility.obj
 0001:000005a5       __onexit                   004015a5 f   MSVCRT:utility.obj
 0001:000005d2       _atexit                    004015d2 f   MSVCRT:utility.obj
 0001:00000634       ___security_init_cookie    00401634 f   MSVCRT:gs_support.obj
 0001:0000067f       ___scrt_exe_initialize_mta 0040167f f   MSVCRT:utility_desktop.obj
 0001:0000067f       ___scrt_initialize_winrt   0040167f f   MSVCRT:utility_desktop.obj
 0001:0000067f       ___scrt_stub_for_initialize_mta 0040167f f   MSVCRT:utility_desktop.obj
 0001:0000067f       __get_startup_commit_mode  0040167f f   MSVCRT:commit_mode.obj
 0001:0000067f       __get_startup_new_mode     0040167f f   MSVCRT:new_mode.obj
 0001:0000067f       __get_startup_thread_locale_mode 0040167f f   MSVCRT:thread_locale.obj
 0001:0000067f       __matherr                  0040167f f   MSVCRT:matherr.obj
 0001:00000682       __get_startup_argv_mode    00401682 f   MSVCRT:argv_mode.obj
 0001:00000686       __get_startup_file_mode    00401686 f   MSVCRT:file_mode.obj
 0001:0000068c       ?__scrt_initialize_type_info@@YAXXZ 0040168c f   MSVCRT:tncleanup.obj
 0001:00000698       ___acrt_initialize         00401698 f   MSVCRT:ucrt_stubs.obj
 0001:00000698       ___acrt_uninitialize       00401698 f   MSVCRT:ucrt_stubs.obj
 0001:00000698       ___scrt_stub_for_acrt_initialize 00401698 f   MSVCRT:ucrt_stubs.obj
 0001:00000698       ___scrt_stub_for_acrt_uninitialize 00401698 f   MSVCRT:ucrt_stubs.obj
 0001:00000698       ___vcrt_initialize         00401698 f   MSVCRT:ucrt_stubs.obj
 0001:00000698       ___vcrt_uninitialize       00401698 f   MSVCRT:ucrt_stubs.obj
 0001:00000698       __should_initialize_environment 00401698 f   MSVCRT:env_mode.obj
 0001:0000069b       __initialize_default_precision 0040169b f   MSVCRT:default_precision.obj
 0001:000006bc       @_guard_check_icall_nop@4  004016bc f   MSVCRT:guard_support.obj
 0001:000006bc       __initialize_denormal_control 004016bc f   MSVCRT:denormal_control.obj
 0001:000006bc       __initialize_invalid_parameter_handler 004016bc f   MSVCRT:invalid_parameter_handler.obj
 0001:000006bf       ___local_stdio_scanf_options 004016bf f i MSVCRT:default_local_stdio_options.obj
 0001:000006c5       ___scrt_initialize_default_local_stdio_options 004016c5 f   MSVCRT:default_local_stdio_options.obj
 0001:000006e2       ___scrt_is_user_matherr_present 004016e2 f   MSVCRT:matherr_detection.obj
 0001:000006ee       ___scrt_get_dyn_tls_init_callback 004016ee f   MSVCRT:dyn_tls_init.obj
 0001:000006f4       ___scrt_get_dyn_tls_dtor_callback 004016f4 f   MSVCRT:dyn_tls_dtor.obj
 0001:000006fa       ___scrt_fastfail           004016fa f   MSVCRT:utility_desktop.obj
 0001:00000815       ___scrt_get_show_window_mode 00401815 f   MSVCRT:utility_desktop.obj
 0001:00000846       ___scrt_initialize_mta     00401846 f   MSVCRT:utility_desktop.obj
 0001:0000084b       ___scrt_is_managed_app     0040184b f   MSVCRT:utility_desktop.obj
 0001:0000088d       ___scrt_set_unhandled_exception_filter 0040188d f   MSVCRT:utility_desktop.obj
 0001:00000899       ___scrt_unhandled_exception_filter@4 00401899 f   MSVCRT:utility_desktop.obj
 0001:000008ef       __crt_debugger_hook        004018ef f   MSVCRT:utility_desktop.obj
 0001:000008f7       __RTC_Initialize           004018f7 f   MSVCRT:initsect.obj
 0001:00000923       __RTC_Terminate            00401923 f   MSVCRT:initsect.obj
 0001:00000950       __SEH_prolog4              00401950 f   MSVCRT:sehprolg4.obj
 0001:00000995       __except_handler4          00401995 f   MSVCRT:chandler4gs.obj
 0001:000009c4       ___isa_available_init      004019c4 f   MSVCRT:cpu_disp.obj
 0001:00000b98       ___scrt_is_ucrt_dll_in_use 00401b98 f   MSVCRT:ucrt_detection.obj
 0001:00000ba4       @__security_check_cookie@4 00401ba4 f   MSVCRT:secchk.obj
 0001:00000bb2       ___raise_securityfailure   00401bb2 f   MSVCRT:gs_report.obj
 0001:00000bda       ___report_gsfailure        00401bda f   MSVCRT:gs_report.obj
 0001:00000cd4       ___current_exception       00401cd4 f   vcruntime:VCRUNTIME140.dll
 0001:00000cda       ___current_exception_context 00401cda f   vcruntime:VCRUNTIME140.dll
 0001:00000ce0       _memset                    00401ce0 f   vcruntime:VCRUNTIME140.dll
 0001:00000ce6       __except_handler4_common   00401ce6 f   vcruntime:VCRUNTIME140.dll
 0001:00000cec       __seh_filter_exe           00401cec f   ucrt:api-ms-win-crt-runtime-l1-1-0.dll
 0001:00000cf2       __set_app_type             00401cf2 f   ucrt:api-ms-win-crt-runtime-l1-1-0.dll
 0001:00000cf8       ___setusermatherr          00401cf8 f   ucrt:api-ms-win-crt-math-l1-1-0.dll
 0001:00000cfe       __configure_narrow_argv    00401cfe f   ucrt:api-ms-win-crt-runtime-l1-1-0.dll
 0001:00000d04       __initialize_narrow_environment 00401d04 f   ucrt:api-ms-win-crt-runtime-l1-1-0.dll
 0001:00000d0a       __get_narrow_winmain_command_line 00401d0a f   ucrt:api-ms-win-crt-runtime-l1-1-0.dll
 0001:00000d10       __initterm                 00401d10 f   ucrt:api-ms-win-crt-runtime-l1-1-0.dll
 0001:00000d16       __initterm_e               00401d16 f   ucrt:api-ms-win-crt-runtime-l1-1-0.dll
 0001:00000d1c       _exit                      00401d1c f   ucrt:api-ms-win-crt-runtime-l1-1-0.dll
 0001:00000d22       __exit                     00401d22 f   ucrt:api-ms-win-crt-runtime-l1-1-0.dll
 0001:00000d28       __set_fmode                00401d28 f   ucrt:api-ms-win-crt-stdio-l1-1-0.dll
 0001:00000d2e       __cexit                    00401d2e f   ucrt:api-ms-win-crt-runtime-l1-1-0.dll
 0001:00000d34       __c_exit                   00401d34 f   ucrt:api-ms-win-crt-runtime-l1-1-0.dll
 0001:00000d3a       __register_thread_local_exe_atexit_callback 00401d3a f   ucrt:api-ms-win-crt-runtime-l1-1-0.dll
 0001:00000d40       __configthreadlocale       00401d40 f   ucrt:api-ms-win-crt-locale-l1-1-0.dll
 0001:00000d46       __set_new_mode             00401d46 f   ucrt:api-ms-win-crt-heap-l1-1-0.dll
 0001:00000d4c       ___p__commode              00401d4c f   ucrt:api-ms-win-crt-stdio-l1-1-0.dll
 0001:00000d52       __initialize_onexit_table  00401d52 f   ucrt:api-ms-win-crt-runtime-l1-1-0.dll
 0001:00000d58       __register_onexit_function 00401d58 f   ucrt:api-ms-win-crt-runtime-l1-1-0.dll
 0001:00000d5e       __crt_atexit               00401d5e f   ucrt:api-ms-win-crt-runtime-l1-1-0.dll
 0001:00000d64       __controlfp_s              00401d64 f   ucrt:api-ms-win-crt-runtime-l1-1-0.dll
 0001:00000d6a       _terminate                 00401d6a f   ucrt:api-ms-win-crt-runtime-l1-1-0.dll
 0001:00000d70       __filter_x86_sse2_floating_point_exception 00401d70 f   MSVCRT:x86_exception_filter.obj
 0001:00000d70       __filter_x86_sse2_floating_point_exception_default 00401d70 f   MSVCRT:x86_exception_filter.obj
 0002:00000000       __imp__UnhandledExceptionFilter@4 00402000     kernel32:KERNEL32.dll
 0002:00000004       __imp__GetCurrentProcess@0 00402004     kernel32:KERNEL32.dll
 0002:00000008       __imp__GetModuleHandleW@4  00402008     kernel32:KERNEL32.dll
 0002:0000000c       __imp__IsProcessorFeaturePresent@4 0040200c     kernel32:KERNEL32.dll
 0002:00000010       __imp__GetStartupInfoW@4   00402010     kernel32:KERNEL32.dll
 0002:00000014       __imp__SetUnhandledExceptionFilter@4 00402014     kernel32:KERNEL32.dll
 0002:00000018       __imp__GetCommandLineA@0   00402018     kernel32:KERNEL32.dll
 0002:0000001c       __imp__QueryPerformanceCounter@4 0040201c     kernel32:KERNEL32.dll
 0002:00000020       __imp__GetCurrentProcessId@0 00402020     kernel32:KERNEL32.dll
 0002:00000024       __imp__GetCurrentThreadId@0 00402024     kernel32:KERNEL32.dll
 0002:00000028       __imp__GetSystemTimeAsFileTime@4 00402028     kernel32:KERNEL32.dll
 0002:0000002c       __imp__InitializeSListHead@4 0040202c     kernel32:KERNEL32.dll
 0002:00000030       __imp__IsDebuggerPresent@0 00402030     kernel32:KERNEL32.dll
 0002:00000034       __imp__TerminateProcess@8  00402034     kernel32:KERNEL32.dll
 0002:00000038       \177KERNEL32_NULL_THUNK_DATA 00402038     kernel32:KERNEL32.dll
 0002:0000003c       __imp____current_exception 0040203c     vcruntime:VCRUNTIME140.dll
 0002:00000040       __imp____current_exception_context 00402040     vcruntime:VCRUNTIME140.dll
 0002:00000044       __imp__memset              00402044     vcruntime:VCRUNTIME140.dll
 0002:00000048       __imp___except_handler4_common 00402048     vcruntime:VCRUNTIME140.dll
 0002:0000004c       \177VCRUNTIME140_NULL_THUNK_DATA 0040204c     vcruntime:VCRUNTIME140.dll
 0002:00000050       __imp__getenv              00402050     ucrt:api-ms-win-crt-environment-l1-1-0.dll
 0002:00000054       __imp____p__environ        00402054     ucrt:api-ms-win-crt-environment-l1-1-0.dll
 0002:00000058       \177api-ms-win-crt-environment-l1-1-0_NULL_THUNK_DATA 00402058     ucrt:api-ms-win-crt-environment-l1-1-0.dll
 0002:0000005c       __imp___set_new_mode       0040205c     ucrt:api-ms-win-crt-heap-l1-1-0.dll
 0002:00000060       \177api-ms-win-crt-heap-l1-1-0_NULL_THUNK_DATA 00402060     ucrt:api-ms-win-crt-heap-l1-1-0.dll
 0002:00000064       __imp___configthreadlocale 00402064     ucrt:api-ms-win-crt-locale-l1-1-0.dll
 0002:00000068       \177api-ms-win-crt-locale-l1-1-0_NULL_THUNK_DATA 00402068     ucrt:api-ms-win-crt-locale-l1-1-0.dll
 0002:0000006c       __imp____setusermatherr    0040206c     ucrt:api-ms-win-crt-math-l1-1-0.dll
 0002:00000070       \177api-ms-win-crt-math-l1-1-0_NULL_THUNK_DATA 00402070     ucrt:api-ms-win-crt-math-l1-1-0.dll
 0002:00000074       __imp___controlfp_s        00402074     ucrt:api-ms-win-crt-runtime-l1-1-0.dll
 0002:00000078       __imp___seh_filter_exe     00402078     ucrt:api-ms-win-crt-runtime-l1-1-0.dll
 0002:0000007c       __imp___set_app_type       0040207c     ucrt:api-ms-win-crt-runtime-l1-1-0.dll
 0002:00000080       __imp____p___argv          00402080     ucrt:api-ms-win-crt-runtime-l1-1-0.dll
 0002:00000084       __imp____p___argc          00402084     ucrt:api-ms-win-crt-runtime-l1-1-0.dll
 0002:00000088       __imp___configure_narrow_argv 00402088     ucrt:api-ms-win-crt-runtime-l1-1-0.dll
 0002:0000008c       __imp__terminate           0040208c     ucrt:api-ms-win-crt-runtime-l1-1-0.dll
 0002:00000090       __imp___get_narrow_winmain_command_line 00402090     ucrt:api-ms-win-crt-runtime-l1-1-0.dll
 0002:00000094       __imp___initterm           00402094     ucrt:api-ms-win-crt-runtime-l1-1-0.dll
 0002:00000098       __imp___initterm_e         00402098     ucrt:api-ms-win-crt-runtime-l1-1-0.dll
 0002:0000009c       __imp__exit                0040209c     ucrt:api-ms-win-crt-runtime-l1-1-0.dll
 0002:000000a0       __imp___exit               004020a0     ucrt:api-ms-win-crt-runtime-l1-1-0.dll
 0002:000000a4       __imp___crt_atexit         004020a4     ucrt:api-ms-win-crt-runtime-l1-1-0.dll
 0002:000000a8       __imp___cexit              004020a8     ucrt:api-ms-win-crt-runtime-l1-1-0.dll
 0002:000000ac       __imp___register_thread_local_exe_atexit_callback 004020ac     ucrt:api-ms-win-crt-runtime-l1-1-0.dll
 0002:000000b0       __imp___initialize_narrow_environment 004020b0     ucrt:api-ms-win-crt-runtime-l1-1-0.dll
 0002:000000b4       __imp___register_onexit_function 004020b4     ucrt:api-ms-win-crt-runtime-l1-1-0.dll
 0002:000000b8       __imp___initialize_onexit_table 004020b8     ucrt:api-ms-win-crt-runtime-l1-1-0.dll
 0002:000000bc       __imp___c_exit             004020bc     ucrt:api-ms-win-crt-runtime-l1-1-0.dll
 0002:000000c0       \177api-ms-win-crt-runtime-l1-1-0_NULL_THUNK_DATA 004020c0     ucrt:api-ms-win-crt-runtime-l1-1-0.dll
 0002:000000c4       __imp____acrt_iob_func     004020c4     ucrt:api-ms-win-crt-stdio-l1-1-0.dll
 0002:000000c8       __imp___set_fmode          004020c8     ucrt:api-ms-win-crt-stdio-l1-1-0.dll
 0002:000000cc       __imp____stdio_common_vfprintf 004020cc     ucrt:api-ms-win-crt-stdio-l1-1-0.dll
 0002:000000d0       __imp____p__commode        004020d0     ucrt:api-ms-win-crt-stdio-l1-1-0.dll
 0002:000000d4       \177api-ms-win-crt-stdio-l1-1-0_NULL_THUNK_DATA 004020d4     ucrt:api-ms-win-crt-stdio-l1-1-0.dll
 0002:000000d8       __imp__JLI_MemAlloc        004020d8     jli:jli.dll
 0002:000000dc       __imp__JLI_GetStdArgs      004020dc     jli:jli.dll
 0002:000000e0       __imp__JLI_GetStdArgc      004020e0     jli:jli.dll
 0002:000000e4       __imp__JLI_CmdToArgs       004020e4     jli:jli.dll
 0002:000000e8       __imp__JLI_Launch          004020e8     jli:jli.dll
 0002:000000ec       \177jli_NULL_THUNK_DATA    004020ec     jli:jli.dll
 0002:000000f0       ___guard_check_icall_fptr  004020f0     MSVCRT:guard_support.obj
 0002:000000f4       ___castguard_check_failure_os_handled_fptr 004020f4     MSVCRT:guard_support.obj
 0002:000000f8       ___xc_a                    004020f8     MSVCRT:initializers.obj
 0002:00000100       ___xc_z                    00402100     MSVCRT:initializers.obj
 0002:00000104       ___xi_a                    00402104     MSVCRT:initializers.obj
 0002:00000110       ___xi_z                    00402110     MSVCRT:initializers.obj
 0002:00000114       ___xp_a                    00402114     MSVCRT:initializers.obj
 0002:00000118       ___xp_z                    00402118     MSVCRT:initializers.obj
 0002:0000011c       ___xt_a                    0040211c     MSVCRT:initializers.obj
 0002:00000120       ___xt_z                    00402120     MSVCRT:initializers.obj
 0002:00000128       ??_C@_04EFFPLJGM@java@     00402128     main.obj
 0002:00000130       ??_C@_07EBOEHGIC@?9J?9ms8m@ 00402130     main.obj
 0002:00000138       ??_C@_0BO@INIJNMDK@?9J?9Djconsole?4showOutputViewer@ 00402138     main.obj
 0002:00000158       ??_C@_0BM@LEDFCKG@sun?4tools?4jconsole?4JConsole@ 00402158     main.obj
 0002:00000174       ??_C@_0BC@INIMDFBD@?1lib?1jconsole?4jar@ 00402174     main.obj
 0002:00000188       ??_C@_0P@MAEHPKDA@?1lib?1tools?4jar@ 00402188     main.obj
 0002:00000198       ??_C@_08BIJCENIG@?1classes@ 00402198     main.obj
 0002:000001a4       ??_C@_07JMAJNDJI@openjdk@  004021a4     main.obj
 0002:000001b4       ??_C@_0BF@FJHGBKOC@_JAVA_LAUNCHER_DEBUG@ 004021b4     main.obj
 0002:000001cc       ??_C@_0BN@NGFJBAGH@Windows?5original?5main?5args?3?6@ 004021cc     main.obj
 0002:000001ec       ??_C@_0BE@OCLPFDNJ@wwwd_args?$FL?$CFd?$FN?5?$DN?5?$CFs?6@ 004021ec     main.obj
 0002:00000200       ??_C@_03LDGAGIDG@1?48@     00402200     main.obj
 0002:00000204       ??_C@_0O@IGGFGIDN@1?48?40_432?9b06@ 00402204     main.obj
 0002:00000220       __load_config_used         00402220     MSVCRT:loadcfg.obj
 0002:00000340       ___safe_se_handler_table   00402340     <linker-defined>
 0002:00000344       ___volatile_metadata       00402344     <linker-defined>
 0002:000006c4       ___rtc_iaa                 004026c4     MSVCRT:initsect.obj
 0002:000006c8       ___rtc_izz                 004026c8     MSVCRT:initsect.obj
 0002:000006cc       ___rtc_taa                 004026cc     MSVCRT:initsect.obj
 0002:000006d0       ___rtc_tzz                 004026d0     MSVCRT:initsect.obj
 0002:00000714       __IMPORT_DESCRIPTOR_jli    00402714     jli:jli.dll
 0002:00000728       __IMPORT_DESCRIPTOR_KERNEL32 00402728     kernel32:KERNEL32.dll
 0002:0000073c       __IMPORT_DESCRIPTOR_VCRUNTIME140 0040273c     vcruntime:VCRUNTIME140.dll
 0002:00000750       __IMPORT_DESCRIPTOR_api-ms-win-crt-stdio-l1-1-0 00402750     ucrt:api-ms-win-crt-stdio-l1-1-0.dll
 0002:00000764       __IMPORT_DESCRIPTOR_api-ms-win-crt-runtime-l1-1-0 00402764     ucrt:api-ms-win-crt-runtime-l1-1-0.dll
 0002:00000778       __IMPORT_DESCRIPTOR_api-ms-win-crt-environment-l1-1-0 00402778     ucrt:api-ms-win-crt-environment-l1-1-0.dll
 0002:0000078c       __IMPORT_DESCRIPTOR_api-ms-win-crt-math-l1-1-0 0040278c     ucrt:api-ms-win-crt-math-l1-1-0.dll
 0002:000007a0       __IMPORT_DESCRIPTOR_api-ms-win-crt-locale-l1-1-0 004027a0     ucrt:api-ms-win-crt-locale-l1-1-0.dll
 0002:000007b4       __IMPORT_DESCRIPTOR_api-ms-win-crt-heap-l1-1-0 004027b4     ucrt:api-ms-win-crt-heap-l1-1-0.dll
 0002:000007c8       __NULL_IMPORT_DESCRIPTOR   004027c8     jli:jli.dll
 0003:00000020       ___scrt_native_dllmain_reason 00403020     MSVCRT:utility.obj
 0003:00000024       ___scrt_default_matherr    00403024     MSVCRT:matherr.obj
 0003:00000030       ___isa_enabled             00403030     MSVCRT:cpu_disp.obj
 0003:00000034       ___security_cookie_complement 00403034     MSVCRT:gs_cookie.obj
 0003:00000038       ___security_cookie         00403038     MSVCRT:gs_cookie.obj
 0003:0000003c       ___scrt_ucrt_dll_is_in_use 0040303c     MSVCRT:ucrt_stubs.obj
 0003:00000040       ___scrt_current_native_startup_state 00403040     MSVCRT:utility.obj
 0003:00000044       ___scrt_native_startup_lock 00403044     MSVCRT:utility.obj
 0003:00000068       ?__type_info_root_node@@3U__type_info_node@@A 00403068     MSVCRT:tncleanup.obj
 0003:00000070       ?_OptionsStorage@?1??__local_stdio_scanf_options@@9@4_KA 00403070     MSVCRT:default_local_stdio_options.obj
 0003:00000078       ___scrt_debugger_hook_flag 00403078     MSVCRT:utility_desktop.obj
 0003:0000007c       ___isa_available           0040307c     MSVCRT:cpu_disp.obj
 0003:00000080       ___favor                   00403080     MSVCRT:cpu_disp.obj
 0003:000003a8       ?_OptionsStorage@?1??__local_stdio_printf_options@@9@9 004033a8     <common>
 0003:000003b0       ___initenv                 004033b0     <common>
 0003:000003b4       ___dyn_tls_dtor_callback   004033b4     <common>
 0003:000003b8       ___dyn_tls_init_callback   004033b8     <common>

 entry point at        0001:0000038c

 Static symbols

 0000:ffffa000       .debug$S                   00400000     vcruntime:VCRUNTIME140.dll
 0000:ffffa000       .debug$S                   00400000     vcruntime:VCRUNTIME140.dll
 0000:ffffa000       .debug$S                   00400000     vcruntime:VCRUNTIME140.dll
 0000:ffffa000       .debug$S                   00400000     vcruntime:VCRUNTIME140.dll
 0000:ffffa000       .debug$S                   00400000     vcruntime:VCRUNTIME140.dll
 0000:ffffa000       .debug$S                   00400000     ucrt:api-ms-win-crt-environment-l1-1-0.dll
 0000:ffffa000       .debug$S                   00400000     ucrt:api-ms-win-crt-environment-l1-1-0.dll
 0000:ffffa000       .debug$S                   00400000     ucrt:api-ms-win-crt-heap-l1-1-0.dll
 0000:ffffa000       .debug$S                   00400000     ucrt:api-ms-win-crt-locale-l1-1-0.dll
 0000:ffffa000       .debug$S                   00400000     ucrt:api-ms-win-crt-math-l1-1-0.dll
 0000:ffffa000       .debug$S                   00400000     ucrt:api-ms-win-crt-runtime-l1-1-0.dll
 0000:ffffa000       .debug$S                   00400000     ucrt:api-ms-win-crt-runtime-l1-1-0.dll
 0000:ffffa000       .debug$S                   00400000     ucrt:api-ms-win-crt-runtime-l1-1-0.dll
 0000:ffffa000       .debug$S                   00400000     ucrt:api-ms-win-crt-runtime-l1-1-0.dll
 0000:ffffa000       .debug$S                   00400000     ucrt:api-ms-win-crt-runtime-l1-1-0.dll
 0000:ffffa000       .debug$S                   00400000     ucrt:api-ms-win-crt-runtime-l1-1-0.dll
 0000:ffffa000       .debug$S                   00400000     ucrt:api-ms-win-crt-runtime-l1-1-0.dll
 0000:ffffa000       .debug$S                   00400000     ucrt:api-ms-win-crt-runtime-l1-1-0.dll
 0000:ffffa000       .debug$S                   00400000     ucrt:api-ms-win-crt-runtime-l1-1-0.dll
 0000:ffffa000       .debug$S                   00400000     ucrt:api-ms-win-crt-runtime-l1-1-0.dll
 0000:ffffa000       .debug$S                   00400000     ucrt:api-ms-win-crt-runtime-l1-1-0.dll
 0000:ffffa000       .debug$S                   00400000     ucrt:api-ms-win-crt-runtime-l1-1-0.dll
 0000:ffffa000       .debug$S                   00400000     ucrt:api-ms-win-crt-runtime-l1-1-0.dll
 0000:ffffa000       .debug$S                   00400000     ucrt:api-ms-win-crt-runtime-l1-1-0.dll
 0000:ffffa000       .debug$S                   00400000     ucrt:api-ms-win-crt-runtime-l1-1-0.dll
 0000:ffffa000       .debug$S                   00400000     ucrt:api-ms-win-crt-runtime-l1-1-0.dll
 0000:ffffa000       .debug$S                   00400000     ucrt:api-ms-win-crt-runtime-l1-1-0.dll
 0000:ffffa000       .debug$S                   00400000     ucrt:api-ms-win-crt-runtime-l1-1-0.dll
 0000:ffffa000       .debug$S                   00400000     ucrt:api-ms-win-crt-runtime-l1-1-0.dll
 0000:ffffa000       .debug$S                   00400000     ucrt:api-ms-win-crt-runtime-l1-1-0.dll
 0000:ffffa000       .debug$S                   00400000     ucrt:api-ms-win-crt-runtime-l1-1-0.dll
 0000:ffffa000       .debug$S                   00400000     ucrt:api-ms-win-crt-runtime-l1-1-0.dll
 0000:ffffa000       .debug$S                   00400000     ucrt:api-ms-win-crt-stdio-l1-1-0.dll
 0000:ffffa000       .debug$S                   00400000     ucrt:api-ms-win-crt-stdio-l1-1-0.dll
 0000:ffffa000       .debug$S                   00400000     ucrt:api-ms-win-crt-stdio-l1-1-0.dll
 0000:ffffa000       .debug$S                   00400000     ucrt:api-ms-win-crt-stdio-l1-1-0.dll
 0000:ffffa000       .debug$S                   00400000     kernel32:KERNEL32.dll
 0000:ffffa000       .debug$S                   00400000     kernel32:KERNEL32.dll
 0000:ffffa000       .debug$S                   00400000     kernel32:KERNEL32.dll
 0000:ffffa000       .debug$S                   00400000     kernel32:KERNEL32.dll
 0000:ffffa000       .debug$S                   00400000     kernel32:KERNEL32.dll
 0000:ffffa000       .debug$S                   00400000     kernel32:KERNEL32.dll
 0000:ffffa000       .debug$S                   00400000     kernel32:KERNEL32.dll
 0000:ffffa000       .debug$S                   00400000     kernel32:KERNEL32.dll
 0000:ffffa000       .debug$S                   00400000     kernel32:KERNEL32.dll
 0000:ffffa000       .debug$S                   00400000     kernel32:KERNEL32.dll
 0000:ffffa000       .debug$S                   00400000     kernel32:KERNEL32.dll
 0000:ffffa000       .debug$S                   00400000     kernel32:KERNEL32.dll
 0000:ffffa000       .debug$S                   00400000     kernel32:KERNEL32.dll
 0000:ffffa000       .debug$S                   00400000     kernel32:KERNEL32.dll
 0000:ffffa000       .debug$S                   00400000     jli:jli.dll
 0000:ffffa000       .debug$S                   00400000     jli:jli.dll
 0000:ffffa000       .debug$S                   00400000     jli:jli.dll
 0000:ffffa000       .debug$S                   00400000     jli:jli.dll
 0000:ffffa000       .debug$S                   00400000     jli:jli.dll
 0001:0000014b       ?pre_c_initialization@@YAHXZ 0040114b f   MSVCRT:exe_winmain.obj
 0001:000001f6       ?post_pgo_initialization@@YAHXZ 004011f6 f   MSVCRT:exe_winmain.obj
 0001:000001fe       ?pre_cpp_initialization@@YAXXZ 004011fe f   MSVCRT:exe_winmain.obj
 0001:00000210       ?__scrt_common_main_seh@@YAHXZ 00401210 f   MSVCRT:exe_winmain.obj
 0001:00000396       ?find_pe_section@@YAPAU_IMAGE_SECTION_HEADER@@QAEI@Z 00401396 f   MSVCRT:utility.obj
 0001:000005e7       ___get_entropy             004015e7 f   MSVCRT:gs_support.obj
 0001:00000950       $$000000                   00401950     MSVCRT:sehprolg4.obj
 0002:000000fc       ?pre_cpp_initializer@@3P6AXXZA 004020fc     MSVCRT:exe_winmain.obj
 0002:00000108       ?pre_c_initializer@@3P6AHXZA 00402108     MSVCRT:exe_winmain.obj
 0002:0000010c       ?post_pgo_initializer@@3P6AHXZA 0040210c     MSVCRT:exe_winmain.obj
 0002:000001ac       _const_cpwildcard          004021ac     main.obj
 0002:000001b0       _const_ergo_class          004021b0     main.obj
 0002:00000214       _GS_ExceptionPointers      00402214     MSVCRT:gs_report.obj
 0002:000006d8       __sehtable$?__scrt_common_main_seh@@YAHXZ 004026d8     MSVCRT:exe_winmain.obj
 0002:000006f8       __sehtable$___scrt_is_nonwritable_in_current_image 004026f8     MSVCRT:utility.obj
 0002:0000091e       .idata$6                   0040291e     jli:jli.dll
 0002:00000a66       .idata$6                   00402a66     kernel32:KERNEL32.dll
 0002:00000acc       .idata$6                   00402acc     vcruntime:VCRUNTIME140.dll
 0002:00000ce8       .idata$6                   00402ce8     ucrt:api-ms-win-crt-stdio-l1-1-0.dll
 0002:00000d08       .idata$6                   00402d08     ucrt:api-ms-win-crt-runtime-l1-1-0.dll
 0002:00000d2a       .idata$6                   00402d2a     ucrt:api-ms-win-crt-environment-l1-1-0.dll
 0002:00000d50       .idata$6                   00402d50     ucrt:api-ms-win-crt-math-l1-1-0.dll
 0002:00000d70       .idata$6                   00402d70     ucrt:api-ms-win-crt-locale-l1-1-0.dll
 0002:00000d92       .idata$6                   00402d92     ucrt:api-ms-win-crt-heap-l1-1-0.dll
 0003:00000000       _const_progname            00403000     main.obj
 0003:00000004       _const_jargs               00403004     main.obj
 0003:00000010       _const_appclasspath        00403010     main.obj
 0003:0000001c       _const_launcher            0040301c     main.obj
 0003:00000048       ?is_initialized_as_dll@@3_NA 00403048     MSVCRT:utility.obj
 0003:00000049       ?module_local_atexit_table_initialized@@3_NA 00403049     MSVCRT:utility.obj
 0003:0000004c       ?module_local_atexit_table@@3U_onexit_table_t@@A 0040304c     MSVCRT:utility.obj
 0003:00000058       ?module_local_at_quick_exit_table@@3U_onexit_table_t@@A 00403058     MSVCRT:utility.obj
 0003:00000088       _GS_ExceptionRecord        00403088     MSVCRT:gs_report.obj
 0003:000000d8       _GS_ContextRecord          004030d8     MSVCRT:gs_report.obj
 0004:00000060       $R000000                   00404060     jconsole.exe.res
